:100000000C94C2020C94FA020C94FA020C94FA02B8
:100010000C94FA020C94FA020C94FA020C94FA0270
:100020000C94FA020C94FA020C949A210C946C220F
:100030000C948E1C0C94FA020C94FA020C94FA02A2
:100040000C94FA020C94FA020C94FA020C94FA0240
:100050000C94FA020C94161D0C94FA020C94FA02F9
:100060000C94FA020C94FA020C94FA020C94FA0220
:100070000C94FA020C94FA020C94FA020C94FA0210
:100080000C94FA020C94FA020C94FA020C94FA0200
:100090000C94FA020C94FA020C94FA020C94FA02F0
:1000A0000C94FA020C94FA020C94FA02BF05BF05F4
:1000B000EB05EB0553067106890789077C061507D2
:1000C00026072607D9220023F8230023F8234C23F0
:1000D0006F23F823C623D52335001E001F00200000
:1000E00021002200230024002500260027002D00E7
:1000F0002E002A002A002B0014001A000800150008
:1001000017001C0018000C00120013002F00300014
:1001100031004C00290004001600070009000A0005
:100120000B000D000E000F003300340028002800E3
:100130004B00E1001D001B00060019000500110026
:100140001000360037003800E500E50052004E0090
:10015000C15CE000E200E30004512C002C000351DC
:10016000E700E600E4000551500051004F00350063
:100170001E001F0020002100220023002400250073
:10018000260027002D002E002A002A002B00140034
:100190001A00090013000A000D000F0018001C00CF
:1001A00033002F00300031004C00290004001500FE
:1001B0001600170007000B00110008000C001200C9
:1001C0003400280028004B00E1001D001B00060041
:1001D000190005000E001000360037003800E50059
:1001E000E50052004E00C15CE000E200E300045173
:1001F0002C002C000351E700E600E40005515000FC
:1002000051004F0035001E001F0020002100220079
:10021000230024002500260027002D002E002A00A0
:100220002A002B0034003600370013001C000900A0
:100230000A00060015000F002F00300031004C00AE
:10024000290004001200080018000C0007000B0031
:100250001700110016003800280028004B00E100AC
:10026000330014000D000E001B00050010001A00E2
:1002700019001D00E500E50052004E00C15CE000E1
:10028000E200E30004512C002C000351E700E600DB
:10029000E4000551500051004F0001003A003B00BE
:1002A0003C003D003E003F00400041004200430052
:1002B000440045000100010001001E021F0220024F
:1002C0002102220223022402250226022702010023
:1002D00001000100490001003A003B003C003D00E4
:1002E0003E003F002D022E022F023002310201009B
:1002F00001000100010040004100420043004400B1
:1003000045000100010001000100010001000100A1
:1003100001000100010001000100010001000100D5
:1003200001000100010001000100010001000100C5
:1003300001003A003B003C003D003E003F00400011
:10034000410042004300440045000100010001005B
:100350001E001F0020002100220023002400250091
:1003600026002700010001000100490001003A00B9
:100370003B003C003D003E003F002D002E002F00C2
:100380003000310001000100010001004000410087
:10039000420043004400450001000100010001004B
:1003A0000100010001000100010001000100010045
:1003B0000100010001000100010001000100010035
:1003C00001000100010053003A003B003C003D00E9
:1003D0003E003F0040004100420043004400450011
:1003E000010001004700680069006A006B006C00B2
:1003F0006D006E006F0070007100720073004800A5
:1004000046003900F500F400F300F200FD00FF00A3
:10041000AB00AA00A900AE00010001000100F90034
:1004200001000100005201520252010001000100CE
:1004300001000100010001000100ED00FA000100CF
:100440000100010001000100F100F10001000100C4
:10045000010001000100EF00EE00F0000E0341007A
:1004600074006F006D006900630000000A034F0014
:100470004C004B00420000000403090409023B0049
:10048000020100A0FA090400000103010100092192
:100490001101000122400007058103080001090441
:1004A00001000103000000092111010001227B006D
:1004B000070582032000011201000200000008ED80
:1004C000FE606001000102000105010902A1018531
:1004D000020901A100050919012908150025019546
:1004E00008750181020501093009311581257F95C3
:1004F000027508810609381581257F9501750881E7
:1005000006050C0A38021581257F950175088106BC
:10051000C0C005010980A101850319012AB7001592
:100520000126B700950175108100C0050C0901A1D5
:1005300001850419012AA002150126A00295017562
:10054000108100C005010906A101050719E029E78E
:100550001500250195087501810295017508810135
:100560000507190029FF150026FF0095067508816B
:100570000005081901290595057501910295017578
:10058000039101C011241FBECFEFDAE0DEBFCDBF63
:1005900004B603FE18C08091820290918302A0915C
:1005A0008402B09185028730904BA740B04B59F43C
:1005B000109282021092830210928402109285029D
:1005C000E0E0F8E3099511E0A0E0B1E0EEEEF9E437
:1005D00002C005900D92A039B107D9F722E0A0E939
:1005E000B1E001C01D92A238B207E1F70E94781372
:1005F0000C94F5240C9400006E9A769A0C942912AF
:1006000081E0089581E008950C94020308950C940C
:1006100006031F93CF93DF9300D000D01F92CDB776
:10062000DEB749835A836B833091930189819A8124
:10063000311114C0662359F0222349F00E94C609E3
:10064000182F682F89819A810E946F0903C00E9428
:100650009A09182F69817A81812F04C00E94C609E6
:1006600069817A810F900F900F900F900F90DF911A
:10067000CF911F910C94FC10FC01262F40815181D9
:100680006281738184810C94090381E00895CF9382
:10069000DF93EC0160E00E943C03BE01DF91CF914B
:1006A0000C9407030C94FC020C94271208950E94EA
:1006B00019080E9456032FEF84E39CE021508040EC
:1006C0009040E1F700C000000C943C1D0F931F9375
:1006D000CF93DF938C0161E00E943C03EC01B801F1
:1006E0000E940403882309F444C0B801CE010E948B
:1006F000FB168823F1F1B801CE010E94591B882313
:10070000C1F1B801CE010E94F617882391F1B8011A
:10071000CE010E94B51A882361F1F80182818823F5
:1007200009F1CB358DE5D807C1F050F4C115FCE5D2
:10073000DF0781F0CF3DDC45A9F40E94F70E19C018
:10074000CC35EDE5DE0761F0CD35DD4559F40E948D
:10075000400E08C00E9457030CC00E94490E02C000
:100760000E944C0EC801DF91CF911F910F910C9404
:10077000000380E0DF91CF911F910F9108950E94B7
:10078000701C80E00E9430170C94DD030E941F163D
:100790000E94E0030C94761C08950C94CC0381E035
:1007A00008950C94CF030895CF93C82F0E94CD03D2
:1007B0008C2F0E94D103CF91089580E00C94D40334
:1007C0000E94B51B0C94D4030E94B51B909192011A
:1007D000891721F0809392010C94D4030895CF934C
:1007E000DF93CDB7DEB72B970FB6F894DEBF0FBE01
:1007F000CDBF4F83588769877A878B8761110E94A5
:100800008C0D9E012F5F3F4F86E0F90111928A9572
:10081000E9F785E0FE013796D90101900D928A959E
:10082000E1F789819A814C815D81452B31F09F3FB1
:1008300031F491E08F3F19F403C091E001C090E0E2
:1008400090FF09C049815A816B817C818D819E8195
:100850000E94AD0C05C0C9010E9445038111F2CF71
:100860002B960FB6F894DEBF0FBECDBFDF91CF91B0
:100870000895FC01808191810E94080A0895CF9318
:10088000882309F4A9C0C82F8238C1F40E94B51B7F
:1008900081FDA2C069E380910201909103010E9451
:1008A000481C0E94AE0D2FEF81EE94E02150804055
:1008B0009040E1F700C0000069E319C0833801F5FA
:1008C0000E94B51B80FD88C063E580910201909174
:1008D00003010E94481C0E94AE0D2FEF81EE94E0B0
:1008E000215080409040E1F700C0000063E5809116
:1008F0000201909103010E944A1CCF910C94AE0D0D
:100900008438C1F40E94B51B82FD66C067E4809103
:100910000201909103010E94481C0E94AE0D2FEF2E
:1009200081EE94E0215080409040E1F700C000004B
:1009300067E4DDCF8CEF8C0F813AF8F48C2F0E94A6
:100940006C1A811149C06C2F8091020190910301B2
:100950000E94121C882349F06C2F80910201909113
:1009600003010E944A1C0E94AE0D6C2F809102016F
:10097000909103010E94481CC0CF80E28C0F883008
:1009800048F4C77081E001C0880FCA95EAF70E9459
:100990006F0DB3CFEBE5EC0FE33040F4F0E0E95B33
:1009A000FE4F808190E0CF910C94DA1BE8E5EC0FCC
:1009B000E73150F4F0E0EE0FFF1FE75EFE4F80815D
:1009C0009181CF910C94F01BCD3E30F08C2F0E9482
:1009D000FD13CF910C94CF14CF910895882309F47F
:1009E00064C0823879F40E94B51B81FF5EC069E360
:1009F00080910201909103010E94481C0E94AE0D5B
:100A000069E310C08338B1F40E94B51B80FF4DC06C
:100A100063E580910201909103010E94481C0E94AD
:100A2000AE0D63E580910201909103010E944A1C82
:100A30000C94AE0D843879F40E94B51B82FF35C04A
:100A400067E480910201909103010E94481C0E947A
:100A5000AE0D67E4E7CF9CEF980F913A10F4682F42
:100A6000E1CF90E2980F983050F4877091E001C088
:100A7000990F8A95EAF7892F0E94750DD9CF9BE5CA
:100A8000980F933020F480E090E00C94DA1B98E506
:100A9000980F973120F480E090E00C94F01B8D3E8D
:100AA00020F00E9458140C94CF1408951F93CF93F4
:100AB000DF93182FEB010E943F04209741F08FE94C
:100AC0009FE00197F1F700C000002197F6CF812F3A
:100AD000DF91CF911F910C94EE04893319F060E0FF
:100AE00070E002C060E570E00C945605882321F0A8
:100AF0000E946F0D0C94AE0D0895882321F00E9482
:100B0000750D0C94AE0D0895CF92DF92EF92FF9287
:100B10000F931F93CF93DF937C01D62FC72FFC0138
:100B20001281058102950F700E94650D8823B9F02E
:100B30001123A9F08C2F807F803421F080E28D0F6B
:100B4000883068F080915B0282FD09C082E00E94DB
:100B50000E0E0E94650D91E0D82ED92601C0D12C31
:100B6000CC2EC2948FE0C8228C2D90E08C30910561
:100B700008F0CFC1FC01EA5AFF4F0C9486248C2F59
:100B8000807FCF70882311F0C295C07F112399F028
:100B9000CC2309F4AAC180E28D0F883010F0D11166
:100BA00004C08C2F0E946F0D03C08C2F0E947F0DFC
:100BB0000E94AE0D9AC18D2F0E94EE04CC2309F441
:100BC000A8C180E28D0F883038F1DD2329F18C2F08
:100BD0000E94850D24C08C2F807FCF70803211F051
:100BE000C295C07FDD2319F0D130A1F13DC08091C5
:100BF0005B0282FF17C0112349F0CC2329F08C2F10
:100C00000E946F0D0E94AE0D80E070C180E00E94D6
:100C1000EE04CC2309F47DC18C2F0E94750D0E9437
:100C2000AE0D77C1112371F0002341F0013031F492
:100C30000E948F0D8C2B0E94970D6BC10E948F0D0F
:100C40008C2B1DC0002319F0013009F462C10E94F1
:100C5000A40D25C0112321F0063008F05AC10EC0A2
:100C6000053008F056C11BC0112361F0002331F09C
:100C7000F701858180FF39C18F7085838C2F0E9499
:100C8000760547C1002359F0D93309F03FC1FFEF82
:100C900007EE13E0F15000401040E1F735C18C2F12
:100CA0000E947D0536C18C2F86958695837019F03C
:100CB000813061F02EC1112321F08D2F9C2F937074
:100CC00002C080E090E00E94DA1B2BC1112321F0CA
:100CD0008D2F9C2F937002C080E090E00E94F01B4B
:100CE00020C18D2F112319F00E94FD1302C00E9414
:100CF00058140E94CF1415C18C2F837009F047C07F
:100D000011110BC12D2F229526952770220F220F2E
:100D10006D2F6F70862F90E0A0E0B0E0022E04C02F
:100D2000880F991FAA1FBB1F0A94D2F7D4FF10C0C7
:100D30004FE050E060E070E004C0440F551F661FB4
:100D4000771F2A95D2F7409550956095709503C00E
:100D500040E050E0BA01C695C695C3708A019B0178
:100D6000082B192B2A2B3B2BC901B801C23049F0A3
:100D700058F4C13019F00E948508CFC00E94730852
:100D8000CCC00E949708C9C00E947108C6C0112338
:100D900019F08C2F817001C08695882309F4BDC09D
:100DA0002D2F229526952770220F220F6D2F6F7001
:100DB000862F90E0A0E0B0E0022E04C0880F991FBB
:100DC000AA1FBB1F0A94D2F7D4FF10C04FE050E017
:100DD00060E070E004C0440F551F661F771F2A951E
:100DE000D2F7409550956095709503C040E050E073
:100DF000BA01C695C695C3708A019B01082B192BB1
:100E00002A2B3B2BC901B801C23049F058F4C1303C
:100E100019F00E944A0981C00E9438097EC00E94D0
:100E20005C097BC00E94AB0878C0CF70112339F0F9
:100E30008C2F0E94D1088D2F0E9476056EC08D2FB9
:100E40000E947D058C2F0E94F20867C0D23F21F1DD
:100E500028F4D03F41F0D13FC1F043C0D33F19F156
:100E6000D43F79F03EC0112341F0053008F051C065
:100E70008C2F8F710E9417094CC0063008F049C0B2
:100E8000F7CF80915B0282FF18C0112339F08C2FBD
:100E90008F710E94D1083DC01123C9F38C2F8F712F
:100EA0000E94F20836C0112329F08C2F8F710E9406
:100EB000BC082FC00E94B7082CC0112349F0CF7185
:100EC0008C2F0E94D10863E08C2F0E94F30D21C06B
:100ED00081E00E940E0E0230E0F082E00E940E0ED1
:100EE00018C0112331F0002391F28D2F0E943F048E
:100EF00010C0002399F2D93349F41FEF27EE33E0F5
:100F0000115020403040E1F700C000008D2F0E94BA
:100F1000EE0488EF8C0D843020F40E94B51B0E94F3
:100F2000D403DD20C9F00E94610D80FD15C0F701DA
:100F300012820E945B0D0E94D108C7010E94CD075A
:100F40000E945B0DDF91CF911F910F91FF90EF9069
:100F5000DF90CF900C94F208DF91CF911F910F9109
:100F6000FF90EF90DF90CF9008950F931F93CF9352
:100F7000DF93EC01688179818A810E94130A8C01D8
:100F80000E946E090E945F08B801CE010E9484058C
:100F9000DF91CF911F910F910895CF93DF93EC01D3
:100FA000988189812B813C81232B31F08F3F31F453
:100FB00081E09F3F19F403C081E001C080E080FD23
:100FC0001DC0CE010E946603811110C00E94650DF4
:100FD0008823A1F08A81882389F080915B0282FDB9
:100FE0000DC082E0DF91CF910C940E0ECE010E94D5
:100FF000B507CE01DF91CF910C944703DF91CF91DC
:10100000089580E090E00E94DA1B80E090E00E946A
:10101000F01B0E948C0D0E94AE0D0E9400160C94D5
:10102000CF1480910201909103010E944C1C0C94FA
:1010300001080E947C0D0C94110892959F709630C7
:1010400079F010F4925001C09A50923068F4803FC9
:1010500069F018F4883E40F409C0843F29F406C0C2
:10106000883E20F0813F11F080E0089581E00895EE
:10107000FC01808191810E94080A0E941D08089548
:10108000CF93DF9300D000D01F92CDB7DEB70F9083
:101090000F900F900F900F90DF91CF910895CF9305
:1010A000DF9300D000D000D0CDB7DEB726960FB6C4
:1010B000F894DEBF0FBECDBFDF91CF9108950895A4
:1010C00008950C9460080C9461080E946308609372
:1010D000CA017093CB018093CC019093CD010C9405
:1010E00001080C9465080F931F930091CA01109199
:1010F000CB012091CC013091CD01602B712B822B43
:10110000932B1F910F910C9465080F931F930091DF
:10111000CA011091CB012091CC013091CD01602307
:101120007123822393231F910F910C9465080F93D1
:101130001F930091CA011091CB012091CC013091F5
:10114000CD0160277127822793271F910F910C945F
:1011500065080C9460080E94A9086093C60170930A
:10116000C7018093C8019093C9010C94010860E005
:1011700070E0CB010C94AB080F931F9341E050E05B
:1011800060E070E08A019B0104C0000F111F221F64
:10119000331F8A95D2F7C901B8011F910F910C94A2
:1011A000AB080F931F9341E050E060E070E004C093
:1011B000440F551F661F771F8A95D2F78091C6018D
:1011C0009091C701A091C801B091C9018A019B010A
:1011D000082B192B2A2B3B2BC901B8011F910F910A
:1011E0000C94AB080F931F9341E050E060E070E077
:1011F00004C0440F551F661F771F8A95D2F740958C
:101200005095609570958091C6019091C701A0910D
:10121000C801B091C9018A019B01082319232A231F
:101220003B23C901B8011F910F910C94AB080F9398
:101230001F9341E050E060E070E004C0440F551F90
:10124000661F771F8A95D2F78091C6019091C701DA
:10125000A091C801B091C9018A019B0108271927F3
:101260002A273B27C901B8011F910F910C94AB08A5
:101270000F931F930091C6011091C7012091C801DF
:101280003091C901602B712B822B932B1F910F91F1
:101290000C94AB080F931F930091C6011091C701E6
:1012A0002091C8013091C9016023712382239323C7
:1012B0001F910F910C94AB080F931F930091C601DF
:1012C0001091C7012091C8013091C9016027712791
:1012D000822793271F910F910C94AB0808952FE05C
:1012E000929F800D1124E82FE695E695E69587708C
:1012F00051E001C0550F8A95EAF785E0E89FF001BB
:101300001124EC56FE4F20E030E070E04081CB012C
:10131000022E02C0969587950A94E2F78170819516
:1013200084278523842781932F5F3F4F2530310504
:1013300069F708952FE0929F800D1124682F66951C
:1013400066956695982F977085E0689FB001112487
:1013500040E050E080E0FB01E40FF51FEC56FE4F4B
:10136000208130E0092E02C0369527950A94E2F7D5
:1013700021703327042E01C0220F0A94EAF7822B32
:101380004F5F5F4F4530510531F70895BF92CF92BF
:10139000DF92EF92FF920F931F93CF93DF938C0115
:1013A000C090C601D090C701E090C801F090C9017B
:1013B0008091CA019091CB01A091CC01B091CD0157
:1013C000C82AD92AEA2AFB2ACFE1D0E0D701C601F0
:1013D0000C2E04C0B695A795979587950A94D2F7D9
:1013E00080FD04C0219790F7B12C07C0BC2EB80136
:1013F0008C2F0E940F110197A9F38B2DDF91CF91B4
:101400001F910F91FF90EF90DF90CF90BF900895C4
:10141000CF93DF93EC010E94C609BE010E940F1119
:10142000DF91CF9108951F93CF93DF93EB019091BC
:101430009301992321F0CB010E94080A13C088234D
:1014400049F0CB010E94C609182F682FCE010E94D7
:101450006F0904C0CB010E949A09182FBE01812F89
:101460000E940F11DF91CF911F9108951F93CF9389
:10147000DF93C091CE0116E08091CF01C81799F09B
:10148000D0E01C9FF0011D9FF00D1124E053FE4F92
:101490004081518162817381848195810E944F08CE
:1014A0002196C770E9CFDF91CF911F9108954091A8
:1014B000000250910102609102027091030280913A
:1014C0000402909105020C944F08EF92FF920F9343
:1014D0001F93CF93DF938091050282958F7009F05F
:1014E00065C080910202882309F460C08091CE011A
:1014F000F090CF011091000200910102609103026F
:101500007091040291E01F3F09F090E0C09100014A
:10151000D0910101292F96E0E92E8F1509F446C0DC
:101520006115710521F00F3F21F030E003C031E07B
:1015300001C0322F90E030FD36C0E89EF001E99EF8
:10154000F00D1124DF01A053BE4F11963C9111976D
:10155000301329C03C91311326C012963C9112974A
:10156000311121C013964D915C911497461B570B76
:101570004C175D07C0F4809105028F7080618093E5
:101580000502EB52FE4F80818F708061808380E086
:1015900092E00E94CD07DF91CF911F910F91FF90B4
:1015A000EF900C94360A01968770B7CFDF91CF91F8
:1015B0001F910F91FF90EF9008959F92AF92BF926D
:1015C000CF92DF92EF92FF920F931F93CF93DF930F
:1015D000CDB7DEB761970FB6F894DEBF0FBECDBFB3
:1015E0008C0185E0F801DE011D9601900D928A952F
:1015F000E1F7D8011296EC9090910002E09101027F
:1016000020910302309104022115310531F0EF3FA2
:1016100031F481E09F3F19F403C081E001C080E014
:10162000B82FB1709B2E80FD47C1D8014C91119607
:101630005C9111971396AD90BC90149780E0C82EE2
:1016400082E0D82EF0900202B501621B730B20914C
:10165000000130910101FF2009F4D9C080910502F9
:101660006217730708F095C0282F207F09F052C039
:101670005E1313C0491311C0FE2CE1100EC08F7011
:101680008061809305020E94570AC6010E94CD071F
:1016900080910502F80185834DC1AB2831F05F3F91
:1016A00031F481E04F3F19F403C081E001C080E0D4
:1016B00080FD03C081E08E2502C080E090E0F82F1D
:1016C000F170FF2E80FF1CC08091CE012091CF01D0
:1016D00036E0821709F40BC190E0389FF001399F82
:1016E000F00D1124E053FE4F6181561306C0608156
:1016F000461303C06281E61203C001968770E9CFEA
:10170000FE2CEE2009F416C18091050281608093C1
:10171000050254C05E1306C0491304C0E11002C0A4
:10172000F80199C0C8010E943808882361F1EE20B1
:1017300051F120910502822F82958F7090E00297DF
:1017400074F0809100029091010298878F8319862E
:10175000BB86AA862C87CE0107960E94CD0786E01D
:10176000F801A0E0B2E001900D928A95E1F70E94A5
:10177000650A0E94570A0AC05E1711F1C8010E944B
:10178000380881112CC0C8010E94CD07FF24F394B2
:10179000D1C0282F207F81F77A2DB98AA88A6E2D93
:1017A00089890E94400880E092E00E94CD0786E08F
:1017B000D6011D928A95E9F70E94570AF12CBAC00A
:1017C0004913DCCFE110DACFF8018583C8010E940C
:1017D000CD0786E0D6011D928A95E9F7ABC0EE20D1
:1017E00091F220910502822F82958F7090E00297EE
:1017F0000CF4B5CF80910002909101029A83898305
:101800001B82BD82AC822E83CE010196A6CF6217C9
:10181000730708F044C0FE2CEE2009F4B4CF5E1329
:1018200030C049132EC02091050220FD21C0822F17
:1018300082958F70482F50E041155105C9F0F8018D
:1018400025834F30510541F08F5F982F9295907FFF
:10185000822F8F70892B8583C8010E94CD0786E077
:10186000F801A0E0B2E001900D928A95E1F73CC04A
:1018700086E0F801A0E0B2E001900D928A95E1F7D0
:1018800059C0C8010E943808811169CF80910502B2
:10189000816080930502C8010E94CD074BC07A2D5C
:1018A000B98AA88A6E2D89890E94400886E0D601EF
:1018B0001D928A95E9F718C0EE2009F464CFC8019B
:1018C0000E943808F82E882309F45DCF86E0F801DD
:1018D000A0E0B2E001900D928A95E1F780E092E0FD
:1018E0000E9439040E94650A0E94570A23C04D874E
:1018F0005E878D859E850E94080A292F22952F706C
:10190000223028F49F7039F0811105C00BC02430BB
:1019100028F49F7049F4805E883020F0C8010E944E
:10192000CD079F2CF92C06C0D80115969C91907F6D
:1019300091F7F8CF8F2D61960FB6F894DEBF0FBEEA
:10194000CDBFDF91CF911F910F91FF90EF90DF906E
:10195000CF90BF90AF909F9008951F93CF93DF9348
:10196000CDB7DEB72C970FB6F894DEBF0FBECDBF54
:101970004F83588769877A878B879C87CE01079624
:101980000E94DD0A8823D1F09F8188852A853B85C6
:10199000232B31F08F3F31F481E09F3F19F403C0D6
:1019A00081E001C080E080FD47C04F815885698596
:1019B0007A858B859C850E944F083EC086E0FE019B
:1019C0003796DE01119601900D928A95E1F7FF811D
:1019D000E8856A857B856115710531F0EF3F31F44B
:1019E00081E0FF3F19F403C081E001C080E080FD89
:1019F00023C02091CF0130E0C9010196877099275B
:101A00004091CE0150E084179507F1F1F983EA8304
:101A10007D836C8396E0929FD001939FB00D11243B
:101A2000A053BE4FFE01319601900D929A95E1F7B9
:101A30008093CF010E94360A16E08091CE019091EA
:101A4000CF01891771F1189FC001112480539E4F57
:101A50000E94DD0A882329F1E091CE011E9FF0014A
:101A60001124E053FE4F4081518162817381848152
:101A700095810E944F088091CE0190E00196877079
:101A800099278093CE01D9CF0E9419081092CF01D7
:101A90001092CE01E0E0F2E086E0DF011D928A952F
:101AA000E9F72C960FB6F894DEBF0FBECDBFDF91DD
:101AB000CF911F91089580910E028595859585950A
:101AC000089580910E028770089590910E0297708C
:101AD00081E009F480E008958091190208959091C1
:101AE0001902892B8093190208958095909119020B
:101AF00089238093190208951092190208959091F4
:101B00001802892B809318020895809590911802ED
:101B100089238093180208951092180208958091E5
:101B20000F02089508950C94920D0C94930D9091CA
:101B30005B0292FD08C090910F02981721F08093EC
:101B40000F020C94950D089580910F02882329F0BF
:101B500010920F0280E00C94950D0895CF93DF93BF
:101B6000E0910201F0910301809119028083E091DC
:101B70000201F0910301908180911802892B8083EA
:101B800080910F02882381F0E0910201F09103011E
:101B90009081892B808380910201909103010E94A2
:101BA000061C81110E94A40DC0910201D091030175
:101BB00048E050E066E072E0CE010E94A624892B46
:101BC00069F088E0FE01A6E0B2E001900D928A95EE
:101BD000E1F7CE01DF91CF910C94C11BDF91CF9142
:101BE00008950C94920D90915B0292FD10C098E0C4
:101BF000899F90011124262B20930E020E94D10868
:101C000080910E028595859585950C94F10D0C9427
:101C1000D10810920E0280E00C94F10D20910E027A
:101C20008095822380930E02982F977099F430E06C
:101C3000482F082E000C550B2417350759F09091AA
:101C40005B0292FD07C08595859585950E94F208F7
:101C50000C94090E089590915B0292FB222720F9C3
:101C6000281769F080FB92F990935B0280915A02E9
:101C700090915B020E94730E82E00C940E0E089508
:101C800080915B0282FB882780F991E089270C9480
:101C90002B0E81E00C942B0E80E00C942B0E80E038
:101CA00090E00E94BB2421E0893E9E4F09F020E095
:101CB000822F089582E090E00C94B32483E090E0BA
:101CC0000C94B324CF9384E090E00E94B324C82FF7
:101CD00082E290E00E94B3242C2F30E0A901582B1F
:101CE000CA01CF910895CF93C92F682F84E090E067
:101CF0000E94C1246C2F82E290E0CF910C94C12409
:101D0000AB01BC018FE090E00C94D324AB01BC018B
:101D100083E190E00C94D32460E070E0CB010C945C
:101D2000860E60E070E0CB010E94800E0C948C0E59
:101D300069EE7EEF80E090E00E94DF2460E082E0C8
:101D400090E00E94C12460E083E090E00E94C12402
:101D50001092CA011092CB011092CC011092CD01C9
:101D600060E084E090E00E94C12460E082E290E0C4
:101D70000E94C12460E085E090E00E94C12460E000
:101D800086E090E00E94C1246FEF87E090E00E941F
:101D9000C12440E050E0BA0188E090E00E94D324E2
:101DA00060E08DE090E00E94C12440E050E0BA0184
:101DB00088E190E00E94D32460E087E190E00E94F7
:101DC000C12440E050E0BA018CE190E00E94D324AD
:101DD00060E070E080E290E00E94DF2440E050E0AC
:101DE000BA0188E190E00E94D3240C94910E0C94E7
:101DF000980E682F8EE090E00C94C1240E94FB1C8A
:101E0000609328027093290280932A0290932B02F8
:101E100060932402709325028093260290932702F8
:101E2000089585B7806885BF85B7806885BF0895A8
:101E300081E008950C94180F08950C941C0F0C94D5
:101E40001C0F0C941F0F0C941C0F0C94230F0C945C
:101E50001C0F0E94110F8BEE91E10E94AB1B0E94A0
:101E6000270F0C94250F0E941D0F0C941C0F0E942D
:101E7000EE110E94D3030C94E6170E94E61C0E9408
:101E8000D1120E94370F0E941F160C94210F5F92EF
:101E90006F927F928F929F92AF92BF92CF92DF927A
:101EA000EF92FF920F931F93CF93DF93CDB7DEB7DF
:101EB0002A970FB6F894DEBF0FBECDBF0E94E61280
:101EC000C82E81110E94FE0E3AE1832E32E0932E3D
:101ED00000E010E0502E802F0E9412125C01F401ED
:101EE000619071904F016826792661147104B1F4F4
:101EF0000F5F1F4F0530110569F78FEF89838A83C4
:101F00001B820E94EF1C8160782F9D838C83498106
:101F10005A816B818D810E94EF033AC080912C021F
:101F200081FD0E941B12D12CEE24E394F12CC301FD
:101F30008E219F21892B29F10E941A0F8823A9F055
:101F4000DE825F82AE20BF2081E0AB2809F480E012
:101F500088870E94EF1C8160782F9A8789874E813D
:101F60005F8168858A850E94EF03000F111FF801C9
:101F7000E65EFD4F80819181E826F926F182E082BC
:101F800007C0D394EE0CFF1CFFE0DF12D0CFB0CF20
:101F900081E0C11001C080E02A960FB6F894DEBF40
:101FA0000FBECDBFDF91CF911F910F91FF90EF90AA
:101FB000DF90CF90BF90AF909F908F907F906F9069
:101FC0005F9008950E94470F0E94E5170E94ED144C
:101FD0000C94E403CF93DF930E941411EC0181155C
:101FE00021E5920708F045C0811530E5930708F018
:101FF00094C0883E910528F5803E910508F0F8C010
:10200000883A910570F4853A910508F07CC08130DA
:10201000910509F475C008F4E8C0049708F0E8C019
:10202000E4C08F3B910508F0E0C0C85AD0E0CC0F67
:10203000DD1FC65BDE4F0990D881C02DCE019464B0
:10204000D8C0811540E2940758F4811551E09507F6
:1020500008F0CEC08D3E910508F4C7C09065C9C098
:10206000C11580E4D80708F4C0C0DF70CE01906AC3
:10207000C0C0811525E59207A8F4811534E59307C2
:1020800008F095C0811543E5940708F07BC08115E1
:1020900052E5950708F061C0D82FCC27CE01816F9B
:1020A000906AA7C0C11589E5D807A0F4C11528E535
:1020B000D20708F082C0C11536E5D30708F095C0F5
:1020C0008C2F0E94A8118F7190E0D82FCC27CE01C1
:1020D00090628FC0C1154AE5D40708F474C0CE01E0
:1020E00090568115904208F080C08D2F8F710E940C
:1020F000A811DD27D0628F71AE01582BCA0179C0BB
:1021000081E090E076C0C55AD0E0C858DE4F8881A3
:10211000C82FD0E0CE0190646CC074E0969587958E
:102120007A95E1F7282F23703C2F337081E090E0FF
:1021300002C0880F991F3A95E2F79C68AC01522BB8
:102140009A019C2F9F709695969550E2959FE0017D
:102150001124C9018C2B9D2B4CC08370992721E041
:1021600030E002C0220F331F8A95E2F79C2F96952C
:10217000969580E2989FE0011124C22BD32BCE01CB
:102180009C6837C08370992721E030E002C0220F9D
:10219000331F8A95E2F79C2F9695969540E2949F7F
:1021A000E0011124C22BD32BCE019A6822C0D82F74
:1021B000CC27CE01846F906A1CC0DC2FCC27CE01C7
:1021C000806F906A16C08C2F8F700E94A81194E0C7
:1021D000D695C7959A95E1F7CF70D0E0DC2FCC2744
:1021E000D0699E01282BC90104C080E090E001C0A5
:1021F000CE01DF91CF9108952BE4829FC00111247D
:10220000FC012FE0729FE00DF11D1124E60FF11D7E
:10221000EE0FFF1FE852FF4F8591949108950E94A1
:10222000FC100E94EA0F08958238910569F1B0F41C
:102230008133910509F46DC048F48932910509F4A0
:1022400063C08A32910509F469C008958533910508
:1022500009F455C089339105B9F00895833E91057D
:1022600069F138F4803E9105B1F0823E910509F1A3
:102270000895863E9105A9F1873E9105B9F1843E06
:10228000910509F064C023C020915A0220FD4FC07F
:1022900021FD4DC0089580915A0280FD44C0809177
:1022A0005B0280FF44C080915A0284FD42C083EEED
:1022B0004DC080915A0282FF38C0F5CF80915A02FA
:1022C00082FD33C080915B0280FD31C0ECCF8091F4
:1022D0005B0281FF32C080915A0284FD2AC087EEE2
:1022E00035C080915A0283FF26C0F5CF80915A02F3
:1022F00083FD21C080915B0281FD1FC0ECCF8091E6
:102300005A0285FD1CC01DC080915A0285FD19C06E
:1023100016C080915A0286FD16C017C080915A02DD
:1023200086FD13C010C089E311C082EE0FC080EE9D
:102330000DC080E00BC086EE09C084EE07C089E2C4
:1023400005C085E303C08AE201C081E390E00895FF
:1023500090915A0292FF0DC0282F2871283019F44D
:10236000877F846006C0282F2471243011F48B7F6E
:10237000886093FF0DC0282F2871283119F4877EBB
:10238000846106C0282F2471243111F48B7E88616A
:1023900020915B0220FF0DC0382F3871383019F4BE
:1023A000877F816006C0382F3171313011F48E7F04
:1023B000886021FF0DC0282F2871283119F4877EED
:1023C000816106C0282F2171213111F48E7E886130
:1023D00094FD877E089580E0089508950E944F0E31
:1023E000811102C00E94F70E0E945A0E80932C02A7
:1023F0000E94620E90935B0280935A020E94ED113C
:102400000E945E0E682F70E080E090E00E947108EC
:102410006091C6017091C7018091C8019091C90176
:102420000C94A908E82FF0E0EE0FFF1FEA59FD4FCA
:10243000808191810895089580EA8A95F1F7089541
:1024400000C008950C941C1208950C9424120C944E
:1024500025120C942412F894E82FE295EF70F0E026
:1024600031A1282F2F7081E090E001C0880F2A95BC
:10247000EAF7982F9095932391A392A1892B82A399
:10248000789408950F931F93CF93DF93CAE8D1E018
:1024900089918F3F11F00E942B1281E0CF38D8072D
:1024A000B9F7CBE7D1E00AE811E089918F3F11F04D
:1024B0000E942B120C171D07C1F7DF91CF911F91BE
:1024C0000F910895BF92CF92DF92EF92FF920F93F8
:1024D0001F93CF93DF938C01C62FD0E0CE01865798
:1024E0009E4F6C01FC0190819F3F09F450C0B62EB5
:1024F000F894E92FE295EF70F0E081A19F7021E060
:1025000030E001C0220F9A95EAF7822B81A382A1C5
:102510002095282322A378940E942012EBE7F1E073
:102520004AE851E021E030E0E12CF12C61916F3F6D
:1025300089F0A62FA295AF70B0E090968C9190E0B4
:102540006F7002C0959587956A95E2F780FD02C08D
:10255000C90102C080E090E0E82AF92A220F331F67
:102560004E175F0719F7F60180818F3F11F00E9427
:102570002B1261E0E114F10409F460E08B2D0E945C
:102580002212CC0FDD1FC00FD11FF982E882DF912C
:10259000CF911F910F91FF90EF90DF90CF90BF9060
:1025A00008950E9442128AE0E6E6F2E0DF01982FE9
:1025B0001D929A95E9F7ECE5F2E0DF011D928A950C
:1025C000E9F785E00E9431130C945203FF920F93B8
:1025D0001F93CF93DF93CDB7DEB72A970FB6F8944A
:1025E000DEBF0FBECDBF8E010F5F1F4F8AE0F80127
:1025F00011928A95E9F7F12C6F2DC8010E946212A1
:10260000F394F5E0FF12F8CF4AE050E0B8018CE512
:1026100092E00E94A624FF24F394009709F4F12C81
:10262000892B41F08AE0F801ACE5B2E001900D920F
:102630008A95E1F72F2D45E066E672E08CE592E0A1
:102640000E9432130E9454038F2D2A960FB6F894DD
:10265000DEBF0FBECDBFDF91CF911F910F91FF90D5
:1026600008950895FF920F931F93CF93DF93F82E51
:10267000092F162FD72FC42F222349F081E08093F2
:102680002F020E94EF1C90932E0280932D028091C6
:102690002F028823D9F080912D0290912E020E9462
:1026A000071D059798F0EF2DF02FA12FBD2F80E08B
:1026B00090E04C2F50E08417950734F4219131912C
:1026C0002D933D930196F7CF10922F02DF91CF917A
:1026D0001F910F91FF9008950E94F21E0E943D0FDE
:1026E0000C94FE1E0E94021F0E94E20F0C941C1FFD
:1026F0000E948D1C0E94D91E0E94290F0E946C13FB
:102700000E9472130E94330FFBCF8091360280FF2C
:1027100006C06091090170E0660F771F26C081FF37
:1027200004C06091090184E005C082FF07C0609188
:10273000090188E0689FB001112417C0909135020B
:102740009923D1F060910801961788F7209109012B
:1027500088E0289F90011124929FA001939F500D23
:10276000112470E0CA010E9450246038710540F4C1
:102770006115710519F406C068E070E0862F0895B0
:102780008FE7089581E008958091360280FF08C0A8
:102790006091050170E0759567957595679521C005
:1027A00081FF06C06091050170E07595679519C0BD
:1027B00082FF04C06091050170E010C09091340266
:1027C000992399F0609104019617A0F78091050173
:1027D000899FC001112470E00E9450246038710567
:1027E00040F46115710519F406C061E070E0862FB0
:1027F00008958FE7089581E008958D3E21F40E94A9
:102800008513819504C08E3E29F40E948513809320
:102810003A0208958F3E21F40E948513819504C0E9
:10282000803F29F40E948513809339020895893FDF
:1028300019F40E94C41305C08A3F31F40E94C413E6
:10284000819580933B0208958B3F21F40E94C4132D
:10285000819504C08C3F29F40E94C41380933C02EC
:1028600008959FE0980F983078F421E030E0A901B6
:1028700002C0440F551F9A95E2F7CA0190913802A1
:10288000892B8093380208958D3F21F48091360280
:1028900081600BC08E3F21F480913602826005C0BA
:1028A0008F3F29F480913602846080933602089528
:1028B0008D3E39F490913A0297FF35C010923A025A
:1028C00059C08E3E29F490913A021916BCF32BC0E0
:1028D000909139028F3E29F497FF25C0109239025A
:1028E00049C0803F19F41916CCF31DC090913B02EA
:1028F000893F29F41916BCF410923B023BC08A3F71
:1029000019F497FF10C0F8CF8B3F39F490913C0237
:1029100097FF09C010923C022DC08C3F21F490918A
:102920003C021916BCF39FE0980F983080F421E028
:1029300030E0A90102C0440F551F9A95E2F7CA0181
:1029400080959091380289238093380213C08D3F7F
:1029500021F4809136028E7F0BC08E3F21F480914E
:1029600036028D7F05C08F3F29F4809136028B7F20
:102970008093360280913902811106C080913A021B
:10298000811102C01092350280913B02811106C074
:1029900080913C02811102C01092340208950E947D
:1029A000EF1C20913902211104C020913A02222308
:1029B00021F0909333028093320220913B02211147
:1029C00004C020913C02222321F090933102809395
:1029D000300287E392E00C94CC1BEF92FF920F93AE
:1029E0001F93CF93DF9300D000D000D0CDB7DEB7D8
:1029F00086E0E7E3F2E0DE01119601900D928A9500
:102A0000E1F7E0903902F0903A0200913B02109118
:102A10003C021092390210923A0210923B0210923C
:102A20003C02E11003C0FF2009F45DC08091320236
:102A3000909133020E94071DAC01909135029923B9
:102A400039F020910A0130E02417350758F04BC0C7
:102A500020910B018AE0289F90011124241735074B
:102A600018F041C09F3F19F09F5F90933502EE2010
:102A700061F00E9485131E1414F09FEF01C091E0D5
:102A8000989F902D112490933902FF2061F00E94AD
:102A900085131F1414F09FEF01C091E0989F902DB3
:102AA000112490933A02309139023323E1F02091BE
:102AB0003A022223C1F045EB3403C00111249923CB
:102AC00019F09093390203C081E08093390235EB0D
:102AD0002303C0011124992319F090933A0203C0F3
:102AE00081E080933A02011103C0112309F45DC013
:102AF00080913002909131020E94071DAC019091AB
:102B00003402992339F02091060130E0241735076B
:102B100058F04BC0209107018AE0289F90011124B2
:102B20002417350718F041C09F3F19F09F5F90931D
:102B30003402002361F00E94C413101614F09FEFBA
:102B400001C091E0989F902D112490933B02112396
:102B500061F00E94C413111614F09FEF01C091E0C0
:102B6000989F902D112490933C0230913B02332387
:102B7000E1F020913C022223C1F045EB3403C00177
:102B80001124992319F090933B0203C081E08093B4
:102B90003B0235EB2303C0011124992319F09093D4
:102BA0003C0203C081E080933C0280913902811194
:102BB0000BC080913A02811107C080913B028111C4
:102BC00003C080913C0281110E94CF14EB82FC82F1
:102BD0000D831E8386E0FE013196A7E3B2E00190EB
:102BE0000D928A95E1F726960FB6F894DEBF0FBED8
:102BF000CDBFDF91CF911F910F91FF90EF9008957E
:102C0000E7E3F2E086E0DF011D928A95E9F7109292
:102C100035021092340210923602089586E090E058
:102C20000C94B324682F86E090E00C94C12480912A
:102C3000700284708961809370020C9412160E9455
:102C40004F0E811104C00E94F70E0E9417160E94B9
:102C50000E1680937002282F26952695269530E033
:102C60002430310524F08770886180937002809150
:102C7000700280FF04C086958695869501C080E02D
:102C80000C94301720917002822F86958695869538
:102C9000482F50E04330510554F48F5F982F990F1F
:102CA000990F990F822F8770892B809370028091E2
:102CB00070028160809370020E94121680917002EF
:102CC0008695869586950C94301780917002982F82
:102CD000969596959695A1F0915E990F990F990FFB
:102CE0008770892B80937002887F91E009F490E0CF
:102CF0008091700290FB80F9809370020E941216FE
:102D0000809170028695869586950C9430178091F7
:102D1000700280FD13C0816080937002813019F4CD
:102D200089E080937002809170020E941216809157
:102D300070028695869586950C943017089580913B
:102D4000700280FF08C08E7F809370020E9412166E
:102D500080E00C94301708958091700280FD0C94EF
:102D60009F160C94871690917002892F86958695F0
:102D700086958F5F8F719770843038F4880F880F35
:102D8000880F892B8093700202C09093700280910B
:102D90007002887F91E009F490E08091700290FBCE
:102DA00080F9809370020E941216809170028695BD
:102DB000869586950C943017843008F083E09091C6
:102DC00070029770282F220F220F220F922B9093C0
:102DD0007002987F21E009F420E09091700220FBBE
:102DE00090F9909370020C9430170E94DC16809139
:102DF00070020C9412169C01FB018281882349F118
:102E00002E3BFCE53F07C9F040F42C3BECE53E07C8
:102E100069F02D3B3C4561F00895203C9CE5390765
:102E200091F070F0213C3C4589F0089583E001C0A9
:102E300080E00E94F51680E008950E946516FBCFA1
:102E40000E944216F8CF0E94AC16F5CF0E94B3162E
:102E5000F2CF81E00895279A2F9808952F9808952A
:102E60008F929F92AF92BF92CF92DF92EF92FF929A
:102E70000F931F93CF93DF93C82F843050F48111A9
:102E800009C080918000877F809380000E942E1768
:102E900006C0C3E080918000886080938000A0918C
:102EA0008600B09187002C2F30E00E948C2423E014
:102EB00030E040E050E00E9464240027122F232FCE
:102EC000342F012F122F232F3327809186009091CA
:102ED00087006CE070E00E943C246017710730F0BE
:102EE000C80169E070E00E943C245EC080918600C9
:102EF00090918700E0908600F0908700E091860036
:102F0000F0918700C6E0D0E0BE010E943C24060F8D
:102F1000171F211D311D4801590185E0880C991C9E
:102F2000AA1CBB1C8A95D1F7C701BE010E943C2494
:102F30006F01E12CF12CA7019601260F371F411DCF
:102F4000511DC501B4010E94642469017A01E09118
:102F50008600F0918700CA01B9010E942C249B01D0
:102F6000AC01DF010E949B249B01AC01C701B601AB
:102F70000E942C24DC01CB012FE0B695A7959795F4
:102F800087952A95D1F7009186001091870020E05F
:102F900030E0081719072A073B0728F460918600DC
:102FA00070918700CB01BC0170938D0060938C0001
:102FB000DF91CF911F910F91FF90EF90DF90CF9015
:102FC000BF90AF909F908F90089508950E942B1707
:102FD0008AE08093800089E1809381008FEF9FEFEA
:102FE00090938700809386000C941F16CF93DF93F5
:102FF000EC01FB018281882309F43CC1C430FDE56A
:10300000DF0760F4CB3F9CE5D90788F49E0122508E
:103010003C452431310508F02EC109C0C236EDE52A
:10302000DE0729F0C63AFDE5DF0709F024C10E945A
:10303000620E90935B0280935A02C1318CE5D807EF
:1030400009F4C6C008F042C0C930ECE5DE0709F457
:103050009BC000F5C5308CE5D80709F485C078F42D
:10306000C330ECE5DE0709F478C008F07AC0C2305E
:10307000DC4509F0F5C080915A028160EFC0C7308D
:103080009CE5D90709F478C008F07AC080915A020B
:103090008061E4C0CD30FCE5DF0709F487C058F457
:1030A000CB309CE5D90709F479C008F07BC080914A
:1030B0005A0288606FC0CF30FCE5DF0709F480C09A
:1030C00008F082C080915A02877FC8C0CE3F9CE53D
:1030D000D90709F471C000F5C531FCE5DF0709F433
:1030E00085C068F4C3319CE5D90709F475C008F0C0
:1030F00095C00E94190880915A028F77AFC0CC3FCB
:10310000FCE5DF07A9F108F054C0CB3FDC4509F02E
:10311000A7C080915B0240C0C230EDE5DE0709F434
:1031200089C058F4C1158DE5D80709F45AC008F0D4
:1031300069C080915B0282602FC0C236EDE5DE0778
:1031400009F47CC0C63AFDE5DF0709F481C0C3304D
:10315000DD4509F085C080E06EC080915A02826032
:103160007DC080915A0216C080915A02886076C054
:1031700080915B0282604FC080915A0280626EC073
:1031800080915A0280646AC00E94190880915A0294
:10319000806864C0846062C081603DC080915A02D2
:1031A0008E7F5CC080915A028D7F58C080915A02F8
:1031B00016C080915B0218C080915B028D7F2BC08E
:1031C00080915A028F7E4AC080915A028F7D46C0FC
:1031D00080915A028F7B42C080915A02877F8B7FF9
:1031E0003DC080915B028D7F8E7F15C080915A0219
:1031F00082FB222720F991E0922790FB82F990FB35
:1032000083F92CC080915B02982F909591708E7FEE
:10321000892B90FB81F980935B0222C00E941908E0
:1032200080915A0287FB222720F991E0922790FB98
:1032300087F914C081E00E94F90E12C080915A02F1
:1032400084FB222720F991E0922790FB84F906C0A5
:1032500080915A02982F909590FB80F980935A02A2
:1032600080915A0290915B020E94730E0E9419088D
:1032700080E001C081E0DF91CF910895893289F12A
:10328000F0F4843171F1B0F4873009F077C081E057
:1032900080930B0184E180930A018AE08093090105
:1032A0008EE18093080188E08093050188E2809395
:1032B000040164C092EE980F9A30F0F05FC0803540
:1032C00009F444C028F48F3409F058C08AE03FC0A4
:1032D000813529F0823509F051C081E038C08FEF87
:1032E00036C080913F02882379F110923F021092FC
:1032F0003E0210923D0242C08D5180933F028330C6
:1033000099F038F4813069F08230D9F48AE091E0A4
:103310000DC0853099F078F0863099F484E091E022
:1033200005C08BE091E002C089E091E090933E02FD
:1033300080933D0223C088E091E0F8CF85E091E0E2
:10334000F5CF10923F021AC080E0089586EFE09119
:103350003D02F0913E02309789F02081082E000C4A
:10336000990B820F911D8F3F910519F014F08FEF8B
:1033700004C097FF02C0108201C0808381E00895DD
:103380000F931F9341E050E060E070E08A019B01E1
:1033900004C0000F111F221F331F8A95D2F7C901E5
:1033A000B8010E9471081F910F910C9419088B317C
:1033B00009F468C058F58B3009F486C078F486307B
:1033C00009F445C020F4853009F44BC07FC0873034
:1033D00009F44AC0883009F477C078C0803109F414
:1033E00064C068F48E3009F071C080912C0282FBB9
:1033F000222720F991E0922790FB82F94CC0863178
:1034000009F462C0893109F45FC060C08A32E1F01A
:1034100060F4873209F455C028F48E3108F456C0A0
:103420008D5150C08932E9F051C0833450F48A3351
:1034300008F045C0853309F444C0883309F444C01A
:1034400045C08334F1F142C00E94F70E3DC0809127
:103450002C02817F8E7F80932C0281E0809340023A
:1034600008950E94570330C080912C02982F9095A8
:10347000917090FB80F980932C02911125C0897F77
:10348000877F10C080912C0281FB222720F991E0D8
:10349000922790FB81F980932C029923A9F08091C7
:1034A0002C02816080932C020FC080912C0283FB40
:1034B000222720F991E0922790FB83F9ECCF8953E2
:1034C00001C080E00E94C01981E0089580E0089565
:1034D00080E008950C94681ACF93C82F8091400221
:1034E000813069F038F08230C1F58C2F0E943E198E
:1034F00081E039C00E946C0D823289F504C00E94BF
:103500006C0D823261F48C2F0E946A1A811104C002
:103510008C2F0E94D7191FC081E090E01CC08C2F17
:103520000E94681A811116C0C43189F058F4CB305A
:1035300089F0C031B1F482E08093400288E30E94B8
:103540003E1908C0C93219F0C83321F00AC01092E0
:10355000400207C081E0817006C01092400280E006
:1035600002C080E0F8CFCF910895CF93DF938631EA
:103570009C4541F5EB010E946C0D982F8A812091AA
:10358000020130910301882379F09A7A81E009F4ED
:1035900080E080934102911102C069E201C065E3BD
:1035A000C9010E94481C0AC080914102811102C0D9
:1035B00069E201C065E3C9010E944A1C0E94AE0D88
:1035C00080E001C081E0DF91CF9108950F931F93B8
:1035D000CF93DF93C42FD22FFC0182818823C9F0BF
:1035E000409344020E94EF1C909343028093420256
:1035F00080E28C0F883008F057C0C77081E001C0AE
:10360000880FCA95EAF7DF91CF911F910F910C9423
:10361000760580914402481330C080914202909117
:1036200043020E94071D883C910538F510E21D0FEA
:10363000CD17B9F080E28C0F883040F4C77081E07C
:1036400001C0880FCA95EAF70E947D05183028F559
:1036500081E09D2F977001C0880F9A95EAF70E942C
:103660007605802F0E946D051830F0F4D77081E048
:1036700001C0880FDA95EAF70AC080E28C0F883023
:1036800098F4C77081E001C0880FCA95EAF7DF910E
:10369000CF911F910F910C947D05802FDF91CF91D9
:1036A0001F910F910C946D05DF91CF911F910F9198
:1036B00008950F939C01CB01243F4CE5340731F171
:1036C00088F4293DFCE53F07D9F02A3D4CE5340755
:1036D00079F1283D3C45A9F506E221EE41EE68ED81
:1036E0007CE52BC0263FFCE53F07E1F0A8F0273F33
:1036F0003C4539F507E225EE46EE67EF7CE51DC057
:1037000007E225EE45EE69ED7CE517C006E221EE05
:1037100040EE64EF7CE511C007E225EE44EE65EF74
:103720007CE50BC006E221EE42EE66EF7CE505C0CB
:1037300008E221E045EE6AED7CE50E94E61A80E0B1
:1037400008C0FC018281882319F01092440201C054
:1037500081E00F91089590939101809390010895D5
:1037600090934A02809349020895E0914902F091B2
:103770004A02309721F00190F081E02D099480E019
:103780000895E0914902F0914A02309721F00280B9
:10379000F381E02D09940895E0914902F0914A02E5
:1037A000309739F022E0DC012C930480F581E02D84
:1037B000099408952091470230914802281739074B
:1037C00071F09093480280934702E0914902F09192
:1037D0004A02309721F00680F781E02D0994089580
:1037E00020914502309146022817390771F09093D5
:1037F000460280934502E0914902F0914A023097D7
:1038000021F00084F185E02D09940895FC013296A1
:1038100097E080E0915029F021912223D9F38F5F26
:10382000F9CF0895662349F0FC013296089621915C
:10383000621729F0E817F907D1F780E0089581E0D1
:1038400008959C01FC0132969FEF80E0419146175C
:1038500089F09F3F19F4411101C0982F8F5F863086
:10386000A9F79F3F39F0F901E90FF11D97FDFA958E
:103870006283089508959C012A5F3F4FFC014281B5
:10388000461301C01282019682179307B9F7089573
:103890000C94211C0C943B1C029626E0FC01119216
:1038A0002A95E9F7089508950C94531C83E08093BA
:1038B0004B020C94541C811102C081E001C082E0D3
:1038C00080934B020C94541C0C945B1C81E08093FD
:1038D0004B020C94541C0C94661C08950C946D1CA3
:1038E0000C946E1C0C946D1C0C946D1C0C946D1C33
:1038F000CF930E94741C0E94E6120E94721CC0E0CA
:103900008C2F0E941212892B29F4CF5FC530C1F78A
:1039100080E001C081E0CF91089508951F920F9239
:103920000FB60F9211248F939F93AF93BF93809103
:103930004C02811113C08091710290917202A0918A
:103940007302B09174024196A11DB11D8093710262
:1039500090937202A0937302B0937402BF91AF91DF
:103960009F918F910F900FBE0F901F90189580918F
:103970007902843031F10E94BF0310924C0220E49E
:1039800088E190E00FB6F894A895809360000FBE90
:103990002093600083B7817F846083BF83B7816099
:1039A00083BF7894889583B78E7F83BF0FB6F894D2
:1039B000A8958091600088618093600010926000FB
:1039C0000FBE08950E9419080C94C60382E084BDBE
:1039D00093E095BD9AEF97BD80936E0008952FB741
:1039E000F8948091710290917202A0917302B0914B
:1039F00074022FBF08952FB7F894609171027091EF
:103A0000720280917302909174022FBF08959C01FD
:103A10004FB7F8948091710290917202A091730255
:103A2000B09174024FBF821B930B089578941F923C
:103A30000F920FB60F9211248F939F93AF93BF9362
:103A40008091710290917202A0917302B091740200
:103A50000196A11DB11D8093710290937202A093F3
:103A60007302B0937402BF91AF919F918F910F90A9
:103A70000FBE0F901F90189581E08093E00080E2C8
:103A80008093D8001092C9008FE19EE40197F1F76E
:103A900000C0000087E090EBDC01809382029093ED
:103AA0008302A0938402B09385029CE088E10FB664
:103AB000F894A895809360000FBE90936000FFCFAC
:103AC000809158020895089522E02093E9002FEF95
:103AD0003091E800215035FD06C035ED3A95F1F7FB
:103AE00000002111F5CF2091E80025FF0BC040E038
:103AF00050E066E070E00E948E1F8091E8008E77B3
:103B00008093E8000895CF93DF9321E02093E900AC
:103B10002FEF3091E800215035FD06C035ED3A9584
:103B2000F1F700002111F5CF2091E80025FF14C026
:103B3000EC0140E050E068E070E00E948E1F809150
:103B4000E8008E778093E80088E0FE01A0E5B2E00F
:103B500001900D928A95E1F7DF91CF9108958093BE
:103B60004D0270934F0260934E028091790284302F
:103B700001F582E08093E9008FEF9091E800815099
:103B800095FD06C095ED9A95F1F700008111F5CFEE
:103B90008091E80085FF0DC040E050E063E070E0F8
:103BA0008DE492E00E948E1F8091E8008E778093D2
:103BB000E8000895BC0184E00C94AF1DBC0183E0D3
:103BC0000C94AF1D80917802811109C00E941F21C1
:103BD0000E947C218091E20084608093E20008953D
:103BE0001092780208950C946B1C6091750281E02C
:103BF000611101C080E00C94561C9091790281E023
:103C0000943009F080E0609175020C945B1C42E0F6
:103C100061EC81E00E94982042E261EC82E00E9427
:103C200098209091790281E0943009F080E06091D1
:103C300075020C94641C80917B02833009F461C08E
:103C400030F4813071F0823009F49AC008958A30DE
:103C500009F486C08B3009F46CC0893009F0A8C023
:103C600020C080917A02813A09F0A2C08091E800D8
:103C7000877F8093E80080917E0290917F02892B5C
:103C800021F468E080E592E003C060E080E090E02D
:103C900070E00E94D91F8091E8008B778093E80044
:103CA000089580917A02813209F082C080917E026B
:103CB00090917F02029708F07BC08091E800877F97
:103CC0008093E8008091E80082FD05C08091790230
:103CD0008111F8CF6DC02091F3008091F20090E047
:103CE000922B029731F48091F100813011F08630EF
:103CF00021F48091F100809358028091E8008B7745
:103D000053C080917A02813A09F052C080917E02BC
:103D100090917F02892B09F04BC08091E800877F4A
:103D20008093E8008091E80080FFFCCF809118012B
:103D300036C080917A028132D9F580917E029091CD
:103D40007F02892BA9F58091E800877F8093E800A6
:103D50000E94CD2080917C02809318010C94190858
:103D600080917A02813221F58091E800877F8093EB
:103D7000E8000E94CD2080917D0280935902089531
:103D800080917A02813AA1F48091E800877F809344
:103D9000E8008091E80080FFFCCF80915902809379
:103DA000F1008091E8008E778093E8000C94CD209C
:103DB000089584B7877F84BF0FB6F894A895809143
:103DC0006000886180936000109260000FBE90E0F8
:103DD00080E80FB6F89480936100909361000FBE65
:103DE0000C94661C0E941F210E947C21E2EEF0E0F0
:103DF00080818460808378940C9411248CE091E01D
:103E00000C94B01B809179028530A9F480917902DD
:103E1000853079F40E94B71C809177028823B1F332
:103E20000E94781C882391F30E94781F0E94190831
:103E3000EDCF0C94E21C089508950C941F1F292FB8
:103E4000332723303105C9F060F42130310581F08A
:103E50002230310509F044C08BE390E02CE734E0D8
:103E600043C021323105E1F02232310549F138C039
:103E700082E190E027EB34E037C09927813091054B
:103E800049F028F0029761F5ECE5F4E005C0E8E7B9
:103E9000F4E002C0ECE6F4E0849190E09F0124C0DD
:103EA0006115710541F061307105D1F489E090E050
:103EB00027EA34E019C089E090E02EE834E014C02D
:103EC0006115710541F06130710551F48BE790E0A7
:103ED00029EC34E009C080E490E024E435E004C03B
:103EE00080E090E020E030E0FA0131832083089503
:103EF00080E189BD82E189BD09B400FEFDCF8091DA
:103F0000D8008F7D8093D8008091E00082608093FC
:103F1000E0008091E00081FDFCCF0895CF92DF9218
:103F2000EF92FF920F931F93CF93DF93EC018B01DE
:103F30007A010E94EC20811133C0E114F10439F0C0
:103F4000F70180819181081B190BC80FD91FC12C63
:103F5000D12C0115110519F18091E80085FD16C0DD
:103F60008091E8008E778093E800E114F10449F035
:103F7000F70180819181C80ED91ED182C08285E06F
:103F80000FC00E94EC20882321F30AC089918093FE
:103F9000F10001501109FFEFCF1ADF0ADACF80E0FC
:103FA000DF91CF911F910F91FF90EF90DF90CF9015
:103FB000089520918002309181022617370748F03A
:103FC0006115710539F42091E8002E772093E800FF
:103FD00001C0B901FC0120E06115710579F1809102
:103FE00079028823F1F18530F1F18091E80083FDB9
:103FF0003CC08091E80082FD2EC08091E80080FFE7
:10400000EBCF2091F3008091F20090E0922B6115AC
:10401000710551F08830910538F421912093F10019
:10402000615071090196F3CF21E0089709F020E073
:104030008091E8008E778093E800CECF2111CFCF1A
:104040000AC080917902882361F0853061F0809107
:10405000E80083FD0AC08091E80082FFF2CF80E093
:10406000089582E0089583E0089581E00895209105
:104070008002309181022617370748F061157105DB
:1040800039F42091E8002E772093E80001C0B901AF
:10409000FC0120E06115710591F18091790288237E
:1040A00009F440C0853009F43FC08091E80083FDE9
:1040B0003DC08091E80082FD2FC08091E80080FF24
:1040C000E9CF2091F3008091F20090E0922B6115EE
:1040D000710559F08830910540F424912093F10046
:1040E0003196615071090196F2CF21E0089709F0ED
:1040F00020E08091E8008E778093E800CBCF2111FB
:10410000CCCF0AC080917902882361F0853061F0BC
:104110008091E80083FD0AC08091E80082FFF2CF21
:1041200080E0089582E0089583E0089581E0089595
:10413000982F973068F59093E900981739F07091AF
:10414000EC002091ED005091F00003C0242F762F59
:1041500050E021FD02C09F5FECCF3091EB003E7F2D
:104160003093EB003091ED003D7F3093ED003091C6
:10417000EB0031603093EB007093EC002093ED0086
:104180005093F0002091EE0027FDE5CF80E00895E8
:104190008F708093E90081E0089580917A0287FF13
:1041A00011C08091E80082FD05C0809179028111E3
:1041B000F8CF11C08091E8008B770BC08091790215
:1041C000882349F08091E80080FFF8CF8091E800D3
:1041D0008E778093E80008952091E4003091E50007
:1041E00095E64091EC00842F817040FF23C08091C0
:1041F000E80080FD1DC080917902882399F0853008
:1042000099F08091EB0085FD11C04091E400509140
:10421000E5002417350729F3915011F09A01E1CFF9
:1042200084E0089582E0089583E0089581E0089590
:1042300080E008954091E80042FFDDCF08950E949C
:104240008D210E949521E0EEF0E0808181608083E5
:10425000E8EDF0E080818F77808319BCA7EDB0E0B6
:104260008C918E7F8C9380818F7E808310927802D8
:1042700008950F931F93CF93DF930E948D210E9487
:104280009521C8EDD0E088818F7788838881806808
:10429000888388818F7D888319BC1092790210925F
:1042A0007502109277021092760200EE10E0F8018B
:1042B00080818B7F808388818160888342E060E099
:1042C00080E00E949820E1EEF0E080818E7F808384
:1042D000E2EEF0E08081816080838081886080836D
:1042E000F80180818E7F8083888180618883DF915F
:1042F000CF911F910F910895E8EDF0E080818F7EBE
:104300008083E7EDF0E080818160808384E082BF7C
:1043100081E0809378020C943921E8EDF0E080810F
:104320008E7F80831092E20008951092DA0010923E
:10433000E10008951F920F920FB60F9211242F9350
:104340003F934F935F936F937F938F939F93AF931D
:10435000BF93EF93FF938091E10082FF0BC08091A8
:10436000E20082FF07C08091E1008B7F8093E10033
:104370000E9410248091DA0080FF1FC08091D80035
:1043800080FF1BC08091DA008E7F8093DA008091DD
:10439000D90080FF0DC080E189BD82E189BD09B4EB
:1043A00000FEFDCF81E0809379020E94E21D05C0EE
:1043B00019BC109279020E94F01D8091E10080FFEB
:1043C00019C08091E20080FF15C08091E2008E7FCD
:1043D0008093E2008091E20080618093E20080910E
:1043E000D80080628093D80019BC85E08093790260
:1043F0000E94F51D8091E10084FF30C08091E200B1
:1044000084FF2CC080E189BD82E189BD09B400FE32
:10441000FDCF8091D8008F7D8093D8008091E100FE
:104420008F7E8093E1008091E2008F7E8093E20096
:104430008091E20081608093E20080917502882380
:1044400011F084E007C08091E30087FD02C081E0A5
:1044500001C083E0809379020E94FD1D8091E100FC
:1044600083FF29C08091E20083FF25C08091E10095
:10447000877F8093E10082E0809379021092750239
:104480008091E1008E7F8093E1008091E2008E7F39
:104490008093E2008091E20080618093E20042E03C
:1044A00060E080E00E9498208091F0008860809316
:1044B000F0000E94F31DFF91EF91BF91AF919F918A
:1044C0008F917F916F915F914F913F912F910F90BD
:1044D0000FBE0F901F9018951F920F920FB60F925C
:1044E00011242F933F934F935F936F937F938F93F9
:1044F0009F93AF93BF93CF93DF93EF93FF93C091BD
:10450000E900CF708091EC00D82FD17080FDD0E809
:104510001092E9008091F000877F8093F0007894FA
:104520000E94B0221092E9008091F0008860809390
:10453000F000CD2BCF70C093E900FF91EF91DF9198
:10454000CF91BF91AF919F918F917F916F915F912B
:104550004F913F912F910F900FBE0F901F90189584
:104560001F93CF93DF93CDB7DEB7AA970FB6F8941A
:10457000DEBF0FBECDBFEAE7F2E08091F10081938C
:1045800022E0E238F207C9F70E941B1E8091E80082
:1045900083FF2EC180917A0290917B02492F50E0D7
:1045A0004A30510508F024C1FA01EE59FF4F0C942E
:1045B0008624803821F0823809F01AC108C0809121
:1045C000760290917702992389F082600FC08091E2
:1045D0007E028F70873008F00BC18093E9008091D4
:1045E000EB0085FB882780F91092E9009091E800A4
:1045F000977F9093E8008093F1001092F100D1C072
:10460000282F2D7F09F0F4C0882319F0823061F043
:10461000EFC080917C02813009F0EAC0933009F04C
:1046200080E0809377022EC080917C0281112AC0A5
:1046300080917E028F702FEF280F263008F0D8C0AF
:104640008093E9002091EB0020FF1CC0933021F4FF
:104650008091EB00806214C09091EB009061909388
:10466000EB0021E030E0A90102C0440F551F8A95FC
:10467000E2F74093EA001092EA008091EB00886034
:104680008093EB001092E9008091E800877F80938F
:10469000E8000E94CD20ACC08111AAC010917C021C
:1046A0001F778091E3008078812B8093E3008091D5
:1046B000E800877F8093E8000E94CD208091E80089
:1046C00080FFFCCF8091E30080688093E3001111AC
:1046D00002C082E001C083E08093790289C08058E3
:1046E000823008F085C080917C0290917D028C3DE3
:1046F00053E0950779F583E08A838AE289834FB78F
:10470000F894DE01139620E03EE051E2E32FF0E062
:1047100050935700E49120FF03C0E295EF703F5F94
:10472000EF708E2F90E0EA3010F0C79601C0C0966F
:104730008D939D932F5F243149F74FBF8091E800FF
:10474000877F8093E8006AE270E0CE0101960E94C4
:10475000D91F16C060917E0270917F02AE014F5F3B
:104760005F4F0E941D1FBC01892B09F441C090912D
:10477000E800977F9093E80089819A810E94372012
:104780008091E8008B778093E80032C0803881F513
:104790008091E800877F8093E80080917502809384
:1047A000F1008091E8008E7772CF811121C0809155
:1047B0007C0290917D0299270297D4F48091E800C1
:1047C000877F8093E80080917C02809375020E942D
:1047D000CD2080917502811106C08091E30087FD94
:1047E00002C081E001C084E0809379020E94071E2C
:1047F0008091E80083FF0AC08091E800877F809362
:10480000E8008091EB0080628093EB00AA960FB6DF
:10481000F894DEBF0FBECDBFDF91CF911F910895F9
:104820000895CF93809179028823A1F0C091E90087
:10483000CF709091EC00892F817090FD80E8C82B9B
:104840001092E9008091E80083FD0E94B022CF70B1
:10485000C093E900CF910895DB018F939F930E944D
:104860009B24BF91AF91A29F800D911DA39F900D9E
:10487000B29F900D11240895AA1BBB1B51E107C0E4
:10488000AA1FBB1FA617B70710F0A61BB70B881FE0
:10489000991F5A95A9F780959095BC01CD0108956F
:1048A00097FB072E16F4009407D077FD09D00E94DD
:1048B0003C2407FC05D03EF4909581959F4F0895C8
:1048C000709561957F4F0895A1E21A2EAA1BBB1B1C
:1048D000FD010DC0AA1FBB1FEE1FFF1FA217B307CC
:1048E000E407F50720F0A21BB30BE40BF50B661FE2
:1048F000771F881F991F1A9469F7609570958095A6
:1049000090959B01AC01BD01CF010895EE0FFF1FF3
:104910000590F491E02D0994A29FB001B39FC001CE
:10492000A39F700D811D1124911DB29F700D811DDB
:104930001124911D08950E948C24A59F900DB49F71
:10494000900DA49F800D911D11240895FB01DC01A1
:1049500004C08D910190801921F441505040C8F756
:10496000881B990B0895F999FECF92BD81BDF89AE5
:10497000992780B50895A8E1B0E042E050E00C949A
:10498000E724262FF999FECF92BD81BDF89A0197B1
:1049900000B4021639F01FBA20BD0FB6F894FA9A87
:1049A000F99A0FBE08950396272F0E94C2240E94F1
:1049B000C124252F0E94C224242F0C94C2240196C6
:1049C000272F0E94C2240C94C124DC01CB01FC01DE
:1049D000F999FECF06C0F2BDE1BDF89A319600B458
:0E49E0000D9241505040B8F70895F894FFCF63
:1049EE00C8001002280850011E0A1401601D831D04
:1049FE00641DDE1DDA1D631D01E200E900EA00B54B
:104A0E0000B600B700CD008301CC008A019201945C
:104A1E00012102230224022502260227022A02B3C2
:104A2E0000B4006F007000818283E200E900EA00AA
:104A3E00B500B600B700CD008301CC008A0192010B
:104A4E0094012102230224022502260227022A02B1
:104A5E00B300B4006F007000818283F1F03067F410
:104A6E00F5F6F794963497939291909535366600B5
:00000001FF
